:10000000003083128A0005280000FF2383168F002A
:10001000003083128A00B9290A108A100A11820757
:1000200007340634043402340A108A100A11820795
:1000300020344D3441344E3425346334203400347C
:100040000A108A100A11820743343A3430343034AB
:10005000323432340A3400340A108A100A1182070A
:1000600049343A3430342534633420344F343A340C
:1000700030342534633400340A108A100A118207A0
:100080002034413433343A34303430342034413441
:1000900034343A342034413435343A34203444341E
:1000A00030343A342034443431343A340A3400346D
:1000B00064005308843C031D5F288A286028A03010
:1000C0000513D5000830D40000008513D50D0513A5
:1000D0000318051700008517D40B6428000085134A
:1000E00000000517732885170000051BD31385131F
:1000F000D31FA02853080739820784288728A028FF
:1001000084288A288F28A028D30A22086128D30AA5
:100110002308612885170517D30AA1306028051721
:10012000000085170830D40085170314051F03103D
:10013000A30D85130517D40B94288517000085138C
:1001400005138517A7200517D31F5828013400343D
:100150000034C410BA01C4183629241AB128640026
:10016000AD28241EB828640005083F06BE04B12847
:100170001630A000A00BBA2800000000D4015408DB
:10018000073C031CE72805083F06BE04640017303F
:10019000A000A00BC92800000000D501241AD50A30
:1001A000000000000000241ED628D50A0000000030
:1001B0000000241EDC28D50A000000000000D5182D
:1001C000E3280310E4280314D30CD40ABF28441CEA
:1001D00004295308213C0319F1285308233C031D2B
:1001E0000329B901253039078400530880004410E1
:1001F0002508233C031D00290430BD0044150329B4
:100200000230BD0044113529B90A3908143C031DD8
:100210000B294414352953080D3C0319132953089D
:100220000A3C031D1629C414441435292530390706
:100230008400530880003D083902031C2D29043036
:100240003D07390203182D293D083902403E84003C
:100250005308000203192D294414441D3529390877
:10026000083C031835295308BA07AB28232A591B21
:100270003E2959080F39A1004329432959080F394C
:10028000093EA100432900345608093C031C4D29AE
:1002900056083038A10052295229093056024038F8
:1002A000A100522900345330840000080319672943
:1002B0000130A100A001A00B5B29A10B5A294A30F3
:1002C000A000A00B612900000000800B5829072B1B
:1002D000A416831605126400831224121F30A00096
:1002E000A00B70290000DC015C08073C031C882976
:1002F0000310DB0C03187E2924127F29241605081D
:100300003F06BE041D30A000A00B8429DC0A74291E
:10031000000000000000000024162030A000A00B08
:100320008F2900000000831605168312A4120034E2
:10033000D81BAA290F30A000570EA0050A302002B2
:100340000318A5293030A007A7295808A0072008BE
:10035000DB0068210F30D7050A3057020318B22995
:100360003030B429D8135808D7075708DB00682164
:1003700000345F30A000213084008001840AA00B8B
:10038000BD292030A000A03084008001840AA00B89
:10039000C529A00184011F30830583169F01801B9E
:1003A0009F0A8312FF2383168F008312DF306500BC
:1003B000A412C801BE010508BF004D30C000413085
:1003C000C1004E30C200A2018330D3005820A108E2
:1003D000031DEB29E4292308073C0318F429A30192
:1003E000A2018030D30058202308C3008430D300FA
:1003F00058202308033C0318042A0330A3000130CB
:10040000A2008030D30058202308C90049080C20DE
:10041000A10083169F0083121F08383941389F00BE
:100420009F30C7004308C707BB013B08073C031CBC
:10043000202A4B303B07840030308000BB0A152A4D
:100440004414C410A9283908C500441D3A2A2608B6
:10045000D9003721210ED400F030D4052708D90067
:10046000372154082104BA074708BA07BA08031904
:100470003A2A222A0530BD073D08BD0A253E8400E0
:100480000008A0005330200203194F2A51302002E7
:100490000319902A433020020319BB2BD32B4908A0
:1004A000033C031D542AD42B02303D07253E840013
:1004B0000008D400D9003721210ED600F030D6052F
:1004C00003303D07253E84000008D800D9003721BD
:1004D00056082104BC0025303D0784000008A00018
:1004E0004F3020020319792A423020020319852A4D
:1004F0008E2A49080C20A100BC053C0885003C0858
:10050000C8003C08BF00BE018F2A49080C20A1008A
:10051000FF3ABC04BC123C0865008F2A8F2AD42BFA
:1005200025303D0784000008433C031DA22A441DDA
:10053000A02AE130BC004308BC07FF30BC06BC0A5F
:100540004A10042B4A14BC01BB0149083B020318A2
:10055000DB2A3B0DA000A00DA00DF830A0051F0860
:10056000C73920049F000630A000A00BB52A000068
:100570001F151F19B92A1E08C6003C08BC0A4B3EAD
:10058000D400460ED5000F30D5055508D6004421BD
:1005900054088400210880003C08BC0A4B3ED4006B
:1005A00046080F39D500D60044215408840021089C
:1005B0008000BB0AA52A05083F06BE043F083E0688
:1005C0000F39BF003F08D60044212108D100480858
:1005D0000739D300D60044212108D200BE01441DB2
:1005E000042B3A30BC004308BC07BB013B08073C66
:1005F000031C012B4B303B0784000008BC07BB0ADF
:10060000F62AFF30BC06BC0A3130D300532924300F
:10061000DB006821441D112B3C08D7003730D8007F
:100620009821D30153081420D30ADB006821043039
:100630005302031D122B4308DB0068212030DB002E
:1006400068214A182E2BD30153082020D30ADB003F
:10065000682107305302031D242BBA2B4930DB00DD
:1006600068213A30DB0068213030DB006821510816
:10067000DB0068210530D30053082C20D30ADB00AF
:10068000682109305302031D3C2B5208DB0068210E
:10069000BC01BB013B08023C031C702B3C08BC0A9C
:1006A0004B3E84000008D4003C08BC0A4B3E84004A
:1006B0000008D6002030DB0068214130DB006821D3
:1006C0003B08D700B730D80098213A30DB006821CA
:1006D0005408DB0068215608DB006821BB0A4A2B5E
:1006E000D30153083C20D30ADB0068210A305302AF
:1006F000031D712B0330D4003030DB006821D40B94
:100700007C2B0A30D50055083C20D50ADB00682137
:100710000E305502031D832B0330D6003030DB0032
:100720006821D60B8E2B0E30D70057083C20D70AF5
:10073000DB00682112305702031D952B0330D800CF
:100740003030DB006821D80BA02B1230D9005908BB
:100750003C20D90ADB00682116305902031DA72B63
:100760000330DA003030DB006821DA0BB22B0A30BC
:10077000DB006821D42B3D08BD0A253E840000081B
:100780000739A30025303D07840000080339BB006A
:10079000A2018030D30058203B08A3008030D30052
:0C07A0005820D12BD42BD42B222A63002C
:02400E000C00A4
:00000001FF
